:1000000000308A00E42A0000FF00030E8301A100F3
:100010000A08A0008A010408A2007708A300780853
:10002000A4007908A5007A08A6007B08A70083131E
:1000300083128C308400801E1F288C1A38288C3044
:100040008400001C25280C183B2822088400230863
:10005000F7002408F8002508F9002608FA00270808
:10006000FB0020088A00210E8300FF0E7F0E09008E
:100070008A110A1265288A110A1232290A108A1076
:100080000A1182075734443454340D340A3400348E
:100090000A108A100A1182070A340D3420344334BE
:1000A000683430343A3425344C34643420340034E9
:1000B00064008C1E58281808ED001A08F800ED1C82
:1000C00063281812181600000034A030700784004E
:1000D0008316E4008312582083166408840078088D
:1000E0008000A030700784000008243C031D7D2898
:1000F0000130F100F0012430A000F10803192D298E
:100100007008043C031D9128043070026F3EE40027
:10011000A030700784000008E500640884006508CA
:1001200080000130F0077008063C03182D29F1010A
:10013000F00101308312EE00831621082F3C0318D2
:10014000A5282108393C0318B5282108403C03188C
:10015000AD282108463C0318B5282108603C031847
:10016000E2282108663C031CE22822082F3C0318E1
:10017000BD282208393C0318CD282208403C03182A
:10018000C5282208463C0318CD282208603C0318E5
:10019000E2282208663C031CE2282208393C0318A6
:1001A000D3280930A2070F30A2052108393C0318D3
:1001B000DB280930A1070F30A1050310210D22040F
:1001C000F200E5288312EB16831625082F3C03184E
:1001D000ED282508393C0318FD282508403C031864
:1001E000F5282508463C0318FD282508603C03181F
:1001F0002A292508663C031C2A2926082F3C0318B7
:1002000005292608393C031815292608403C0318FF
:100210000D292608463C031815292608603C0318BA
:100220002A292608663C031C2A292608393C03187B
:100230001B290930A6070F30A6052508393C0318ED
:1002400023290930A5070F30A5050310250D260425
:10025000F3002D2983126B17831683128C128A11D7
:100260000A122528D70B3E290130CF070318D00AE0
:100270000319D10A0319D20A0F30D7000C108A11C2
:100280000A1225287508840083165C088000840AF9
:100290008001F50A831200348316DB1B61290F30BD
:1002A000F7005A0EF7050A30770203185A29303042
:1002B000F7075C295B08F7077708DC008312422107
:1002C00083160F30DA050A305A02031869293030D4
:1002D0006B29DB135B08DA075A08DC008312422122
:1002E0008A110A12BA2983160612831206120034E2
:1002F0008C1E7C295820782900348316061283121C
:1003000006160C1E812983166208831299000000CC
:1003100083160612831206168316981891298312E3
:100320008C290612831206120034E1308400000882
:100330000319AB290130F800BF30F7006400F70B58
:100340009E29F80B9C294A30F700F70BA5290000DD
:100350006400800B9A290034C630F5003F308316C4
:10036000DC00831242216C088316DA005730DB0070
:1003700083124C2920308316DC0083124221C630C0
:100380008316DA004408DB001030DC005A08DD0078
:100390005D08840080080319CF29DD0AC8295B089D
:1003A000840080080319E4295C08003C0318E42950
:1003B0005B0884000008DF005D0884005F0880009F
:1003C000DD0ADB0ADC03CF295D08840080015A08BE
:1003D000F8007808C400C501440845078400800877
:1003E0000319F429C50AEC29DA0183127321831653
:1003F000DC01DB015C08013C031C1C2A031D042AF0
:100400005B08903C031C1C2AF417740887008312B5
:10041000871B0F2A8316DC01DB01152A8312640077
:100420001030F700F70B122A8316DA08031D640058
:10043000DB0A0319DC0AFA29831278216C08831677
:10044000DA004508DB004408DC00601083127321E9
:100450008316DD015D08043C031C552A83126D13CD
:100460008316DE015B085E020318412A5C088400E3
:100470000008E100E20083127D218316DC0ADE0A17
:10048000322A83126D1B4D2A4E088316E100831217
:10049000952183166014552A83124E088316E100B5
:1004A000831295218316DD0A2A2A831278210030CF
:1004B000831660180130F800F808031D652A0A3019
:1004C000E100831295211E2A831683128A110A12D3
:1004D000922B04088316CC00C61F762ACC174C1E1C
:1004E000CC0AC509C609C50A0319C60A460EF03862
:1004F000C800C807E23EC900323ECB0046080F39AB
:10050000C907C907CB07E93ECA00CA07CA07450E93
:100510000F39CA07CB07CA0DCB0DCB09CB0D450848
:100520000F39CB07C80D0730C7000A30CB07CA0305
:10053000031C962ACA07C903031C9A2AC907C803C1
:10054000031C9E2AC807C703031CA22AC7308400C5
:1005500007304C054C1384034C05031DB62A4C1A76
:10056000840A4C1AB62A2030F700D32A8407CB30ED
:10057000040203194C170008F700031DC72A4C1B7F
:10058000C72A4C1ADD2ACC19C72A2030D22ACC1F00
:10059000CF2A2D30F70084034C13CC13D32ACC156B
:1005A0004C123030F707C6010408C5007708E20096
:1005B00083127D21831645088400840A4C1FB72AC4
:1005C00083128A110A12F92B84011F3083058316C6
:1005D00006128312061219308316990026309800ED
:1005E00090308312980083161F149F141F159F11BB
:1005F00007309C008312A9010130AA00AB01AC01B5
:10060000AD014630AE00AF015130B000B101533002
:10061000B200B3015630B400B5014130B600B701A5
:100620005230B800B9010330CE00CF01D001D10162
:10063000D201D301D401D501D601D701D801D90106
:10064000DA01DB01DC01DD01DE01DF01E001E101B6
:10065000E201E301E401E501E601E701E801E90166
:10066000EA016B10EB106B11EB116B12EB126B13B9
:10067000EB13EC01ED01F101FF30F200F301F400A6
:10068000F501F601FC01FD01FE01831640100F305B
:100690008312D7000C30F7000730810181308400CD
:1006A0000008F0390738800064000008F739F719AE
:1006B000F0397704800083161F1383121F179F17CA
:1006C00083169F1783121F1483161F109F101F116C
:1006D0009F1503081839F7000E08033977040E1424
:1006E0008E14831503160B3A831203197B2B133ACE
:1006F0000319912B922B3A30F5008316C40144085C
:1007000083123E208316C40AF700DC0083124221C4
:10071000053083164402031D7F2B3A30C400831238
:10072000AC29922B8316C3012030F80083121F08D6
:10073000C73978049F0064008C1EAB2B58208316A9
:10074000C3080319A52B0030A62B0130C3002130AC
:10075000E20083127D218316C3080319BF2B831285
:100760008714F4107408831687000430C400FA302C
:10077000E100831295218316C40BB72BCE2B831275
:100780008710F4107408831687000430C400FA3010
:10079000E100831295218316C40BC72B0430C400DB
:1007A000FA30E100831295218316C40BD02B8312FB
:1007B0001F151F19D92B1E08FA0083161E08C10029
:1007C0007A08C200C4014408831248208316C40A70
:1007D000F700E20083127D21073083164402031DD7
:1007E000E32B103084004208C6004108C500831284
:1007F000692A20308316E20083127D219B2B63003F
:02400E00753FFC
:00000001FF
